:020000020000FC
:10000000E3E0EEBFE0E0EDBF239A539A559A229ABF
:10001000549A219A579A3B9A3DD1EF93FF93E8EE79
:10002000F3E0EF93FF93ECECF7E03197F1F7FF91FA
:10003000EF91319711F000C0F4CFEF91FF915EE1A5
:100040005F9A439AE52F5C9A299A2B9AEF93FF9334
:10005000E4E0F0E0EF93FF93ECECF7E03197F1F799
:10006000FF91EF91319711F000C0F4CFEF91FF9124
:100070002B98EF93FF93ECE0F0E0EF93FF93ECEC21
:10008000F7E03197F1F7FF91EF91319711F000C050
:10009000F4CFEF91FF91EA9509F0D5CF2B985C98BA
:1000A00029985F984398E52F299A2B9A5B9AEF93AA
:1000B000FF93E4E0F0E0EF93FF93ECECF7E031978F
:1000C000F1F7FF91EF91319711F000C0F4CFEF916C
:1000D000FF912B985B98EF93FF93ECE0F0E0EF93A8
:1000E000FF93ECECF7E03197F1F7FF91EF91319747
:1000F00011F000C0F4CFEF91FF91EA9509F0D4CF51
:1001000029982B985B985F9A439AE52F2A9A299A07
:100110005B9AEF93FF93E4E0F0E0EF93FF93ECEC56
:10012000F7E03197F1F7FF91EF91319711F000C0AF
:10013000F4CFEF91FF915B98EF93FF93ECE0F0E049
:10014000EF93FF93ECECF7E03197F1F7FF91EF912C
:10015000319711F000C0F4CFEF91FF91EA9509F0CB
:10016000D5CF29982A985B985F984398E52F2A9ACB
:100170005B9A5D9AEF93FF93E4E0F0E0EF93FF93D7
:10018000ECECF7E03197F1F7FF91EF91319711F037
:1001900000C0F4CFEF91FF915B985D98EF93FF93D0
:1001A000ECE0F0E0EF93FF93ECECF7E03197F1F740
:1001B000FF91EF91319711F000C0F4CFEF91FF91D3
:1001C000EA9509F0D4CF2A985B985D985F9A439A94
:1001D000E52F2A9A5C9A5D9AEF93FF93E4E0F0E0B2
:1001E000EF93FF93ECECF7E03197F1F7FF91EF918C
:1001F000319711F000C0F4CFEF91FF915D98EF932C
:10020000FF93ECE0F0E0EF93FF93ECECF7E0319735
:10021000F1F7FF91EF91319711F000C0F4CFEF911A
:10022000FF91EA9509F0D5CF2A985C985D985F9880
:100230004398E52F5C9A2B9A5D9AEF93FF93E4E045
:10024000F0E0EF93FF93ECECF7E03197F1F7FF91DB
:10025000EF91319711F000C0F4CFEF91FF912B98FF
:100260005D98EF93FF93ECE0F0E0EF93FF93ECECFD
:10027000F7E03197F1F7FF91EF91319711F000C05E
:10028000F4CFEF91FF91EA9509F0D4CF2B985C98C9
:100290005D98D6CE5F9AEF93FF93E8EEF3E0EF938D
:1002A000FF93ECECF7E03197F1F7FF91EF91319785
:1002B00011F000C0F4CFEF91FF91439AEF93FF93B9
:1002C000E8EEF3E0EF93FF93ECECF7E03197F1F712
:1002D000FF91EF91319711F000C0F4CFEF91FF91B2
:1002E0004398EF93FF93E8EEF3E0EF93FF93ECEC8A
:1002F000F7E03197F1F7FF91EF91319711F000C0DE
:0A030000F4CFEF91FF915F9808958C
:00000001FF
